:020000040000FA
:0400000004303A2866
:08000800A000030EA100831209
:1000100005191028831601178312B23081002B288E
:1000200083160113831203140B190310A80DA90DD5
:10003000AA0DAB0DAC0DAC16FF302C02031D2B2806
:10004000FA302B02031D2B2831152A08AF0029088E
:10005000AE002808AD008B100B11210E8300A00EFE
:04006000200E090065
:0C007400203084008001840A6030040207
:10008000031C3C281230B0006B218316FF23900024
:10009000831283160C308505870183128501870141
:1000A000073099000030831691009F008312C830FA
:1000B00083168100831231309000003083168C004B
:1000C000831210308B00C52181018E018F010B112D
:1000D0008B100B108C018B177B2031197E20B30BFA
:1000E0007928031085190314B90DF030390203196A
:1000F000EE20C6216C286400321008003111013056
:10010000B7008B132030370783169B001C141A0886
:100110008312A4001030370783169B001C141A08A2
:100120008312A300A6000230A6060030370783160C
:100130009B001C141A088312A200A7000130A70616
:100140008B17321CA92822090339A200A309A4098C
:10015000A50924082F02031DE82823082E02031DE9
:10016000CA2822082D02031DE82801303702031D8A
:10017000BC283D143E14792102303702031DC328E8
:10018000BD143E14852103303702031DCA283D15D6
:100190003E14912126082E02031DE82827082D026F
:1001A000031DE82801303702031DD9283D103E14F5
:1001B0009D2102303702031DE028BD103E149E2110
:1001C00003303702031DE7283D113E149F21E82824
:1001D000B70A043037020318080081280130B6003E
:1001E000B300B400B500B70085018701B113B42195
:1001F0007B20B30B1B29031085190314B90DF030B4
:10020000390203194229B41F8501B41F8701B40BB9
:100210001B29B50B1B290230B50001303702031929
:10022000A021023037020319A52103303702031938
:10023000AF21FA30B400311DF8283111321C2529C4
:100240002D090339AD00AE09AF092F1CF8288E0126
:100250008F010C1CF8280C102E1EF8288B13203050
:100260003707BB002F08BA00582110303707BB00F2
:100270002E08BA00582100303707BB002D08BA00FD
:1002800058218B17B72185018701B70AB6010430C1
:100290003702031CF828C0010800C52108003E1CD5
:1002A00008003E101030BB003D08BA00582108007D
:1002B0008B133A0883161C159A003B089B00553097
:1002C0009D00AA309D009C1464009C1864291C1198
:1002D00083128B170800831620309B001C141A0809
:1002E0008312C2000130C21BC200C2080319C2003F
:1002F00008008516051285100510C001C0148E0176
:100300008F010C104208C1000800851605128510E7
:100310000510C00140158E018F010C104208C1006C
:1003200008008512051285140510C001C0158E0144
:100330008F010C104208C1000800080008000800E6
:10034000380903398500B8000800C00A3809333974
:10035000B800C01C0339C0183039850008003809BE
:1003600030398500B8000800B801B8140800B80199
:1003700001303702031DBE29B81438160230370287
:10038000031DC4290000B816080008000C1C6C28C6
:100390000C10C10B6C284208C1008501C01805145F
:1003A00040198514C0190516C0018E018F010C106B
:0603B0004208C100080034
:084000000300030005000800A5
:02400E00CC01E3
:10420000010078007A007C007E007B0079007F004E
:104210007D007A0078007E007C00FF00FF00FF0038
:104220000000F200F600FA00FE00F200F600FA00CC
:10423000FE00F200F600FA00FE00FF00FF00FF00A3
:10424000010005000500050005000900090009003E
:1042500009000D000D000D000D00FF00FF00FF0024
:10426000FF00FF00FF00FF00FF00FF00FF00FF0056
:10427000FF00FF00FF00FF00FF00FF00FF00FF0046
:10428000FF00FF00FF00FF00FF00FF00FF00FF0036
:10429000FF00FF00FF00FF00FF00FF00FF00FF0026
:1042A000FF00FF00FF00FF00FF00FF00FF00FF0016
:1042B000FF00FF00FF00FF00FF00FF00FF00FF0006
:1042C000FF00FF00FF00FF00FF00FF00FF00FF00F6
:1042D000FF00FF00FF00FF00FF00FF00FF00FF00E6
:1042E000FF00FF00FF00FF00FF00FF00FF00FF00D6
:1042F000FF00FF00FF00FF00FF00FF00FF00DD00E8
:00000001FF
